:020000040000FA
:10000000F8EF16F0C96E1200F5EF09F0ACA2FED7BA
:10001000AD6E1200C28212000DEF11F0D9CFE5FFD4
:10002000E1CFD9FF00C0E5FF01C0E5FF02C0E5FF59
:1000300003C0E5FF04C0E5FF05C0E5FF06C0E5FF1E
:1000400007C0E5FF08C0E5FF09C0E5FF0AC0E5FFFE
:100050000BC0E5FF0CC0E5FF0DC0E5FF0EC0E5FFDE
:100060000FC0E5FF10C0E5FF11C0E5FF12C0E5FFBE
:1000700013C0E5FF14C0E5FF15C0E5FF16C0E5FF9E
:1000800017C0E5FF18C0E5FF19C0E5FF1AC0E5FF7E
:100090001BC0E5FF1CC0E5FF1DC0E5FF1EC0E5FF5E
:1000A000020EDBCF00F0030EDBCF01F0040EDBCF3E
:1000B00002F0050EDBCF03F0060EDBCF04F0070ED7
:1000C000DBCF05F0080EDBCF06F0090EDBCF07F023
:1000D0000A0EDBCF08F0096A0A6A02C00DF00D5063
:1000E000800A0DE102500801026F0150016F0050BB
:1000F000006F080E016E000E006E800E026E03C0CF
:10010000E9FF04C0F3FF0550B5EC16F00B6E0B5081
:10011000D8B4CAEF03F00B50250A02E0B1EF03F0A8
:100120000C6A0D6A0E6A0F6A106A0A0E116E126A64
:10013000136A146A200E156E1668176A2B0E186E55
:10014000032A02E3044A052A03C0E9FF04C0F3FFBF
:100150000550B5EC16F0196E250A13E11950E56E3D
:100160000250E56E0150E56E0050E56E49EC0EF070
:10017000040EE126094A0A2A032A02E3044A052A50
:10018000BED71950300A06E1300E156E032A02E37D
:10019000044A052A03C0E9FF04C0F3FF0550B5EC8B
:1001A00016F02D0A06E1010E146E032A02E3044A3A
:1001B000052A03C0E9FF04C0F3FF0550B5EC16F0B3
:1001C000200A08E1010E176E200E186E032A02E3C2
:1001D000044A052A03C0E9FF04C0F3FF0550B5EC4B
:1001E00016F02B0A06E1010E176E032A02E3044AF9
:1001F000052A03C0E9FF04C0F3FF0550B5EC16F073
:10020000196E800F4F0F2DE31950800F460F29E212
:1002100003C019F004C01AF005C01BF019C0E9FFB3
:100220001AC0F3FF1B50B5EC16F01C6E800F500F78
:1002300012E31C50800F460F0EE213500A0DF3CF4D
:100240001DF01D501C26D00E1C24136E192A02E32B
:100250001A4A1B2AE3D719C003F01AC004F01BC0C6
:1002600005F003C0E9FF04C0F3FF0550B5EC16F03C
:100270002E0A2EE1032A02E3044A052A166A03C065
:1002800019F004C01AF005C01BF019C0E9FF1AC02C
:10029000F3FF1B50B5EC16F01C6E800F500F12E3ED
:1002A0001C50800F460F0EE216500A0DF3CF1DF0C2
:1002B0001D501C26D00E1C24166E192A02E31A4A61
:1002C0001B2AE3D719C003F01AC004F01BC005F0C5
:1002D00003C0E9FF04C0F3FF0550B5EC16F0196E3A
:1002E0006C0A07E1010E0C6E032A02E3044A052A98
:1002F00009D01950680A06E1010E0E6E032A02E3C6
:10030000044A052A03C0E9FF04C0F3FF0550B5EC19
:1003100016F0750A06E1010E106E032A02E3044A84
:10032000052A03C0E9FF04C0F3FF0550B5EC16F041
:10033000196E730A05E1010E0D6E200E156E3FD089
:100340001950780A03E1100E116E39D01950580A6D
:1003500005E1100E116E010E126E31D01950630AB4
:1003600002E1116A2CD019506F0A03E1080E116ED8
:1003700026D01950660A03E1010E0F6E20D01950E5
:10038000640A1DE01950690A1AE0105005E0FF0EDA
:1003900003260422052213D01950E56E0250E56EA3
:1003A0000150E56E0050E56E49EC0EF0040EE126BA
:1003B000094A0A2A032A02E3044A052AA0D60D5054
:1003C00021E00650030F0D6E000E0720196E000E7F
:1003D00008201A6E0DC006F019C007F01AC008F008
:1003E000FD0E0D26FF0E19221A220DC0E9FF19C0BD
:1003F000F3FF1A5087EC15F00D6EF3CF19F0F4CF20
:100400001AF000D10F500DE0000E1A6E080E196E92
:100410001C0E0D6E040E0626000E0722082216681A
:10042000F1D016680C5023E00650040F0C6E000E3D
:1004300007200F6E000E08201B6E0CC006F00FC0C8
:1004400007F01BC008F0FC0E0C26FF0E0F221B222B
:100450000CC0E9FF0FC0F3FF1B502BEC14F00C6E27
:10046000F3CF0FF0F4CF1BF0E9CF1CF06AD00E50A1
:1004700032E00650020F0E6E000E07201D6E000EB9
:1004800008201E6E0EC006F01DC007F01EC008F04A
:10049000FE0E0E26FF0E1D221E220EC0E9FF1DC0FD
:1004A000F3FF1E5003EC16F00E6E0EC00CF0E86A5F
:1004B0000EBEFF0E0F6E1B6E1C6E11500A0A03E17A
:1004C0001050D8B43ED00C500E6E0EC00CF00F6A17
:1004D0001B6A1C6A36D00650020F0E6E000E0720F3
:1004E0001D6E000E08201E6E0EC006F01DC007F027
:1004F0001EC008F0FE0E0E26FF0E1D221E220EC08C
:10050000E9FF1DC0F3FF1E5003EC16F00E6EF3CF93
:100510001DF00EC00CF01DC00FF0E86A1DBEFF0EEE
:100520001B6E1C6E11500A0A02E110500AE00C50BA
:100530000E6E0F501D6E0EC00CF01DC00FF01B6A2A
:100540001C6A0F0E196E420E0D6E800E1A6E11503F
:10055000D8B440D0105013E01150E56E0F0EE56E88
:10056000420EE56E1C50E56E1B50E56E0F50E56EB9
:100570000C50E56E19EC09F0070EE12612D011506F
:10058000E56E0F0EE56E420EE56E1C50E56E1B50DB
:10059000E56E0F50E56E0C50E56E54EC0FF0070E53
:1005A000E12617502FE00DC0E9FF19C0F3FF1A50E4
:1005B000B5EC16F02D0A26E0FF0E0D2619221A22A0
:1005C00018C0E5FF0DC0E9FF19C0F3FF1A50E3ECB6
:1005D00016F018D00CC0E5FF0DC0E9FF19C0F3FFFD
:1005E0001A50E3EC16F00D50010F0C6E000E19209E
:1005F0000E6E000E1A20E56A0CC0E9FF0EC0F3FF74
:10060000E3EC16F00DC00CF019C00EF01AC00FF09C
:1006100013C010F0105010E00CC0E9FF0EC0F3FF43
:100620000F50B5EC16F0176E175006E00C2A02E3D7
:100630000E4A0F2A1006EED710C013F014501EE118
:1006400009C00CF00AC00EF010C00FF00F5010E0FF
:100650001550E56E0250E56E0150E56E0050E56EF6
:1006600049EC0EF0040EE1260C4A0E2A0F06EED7D6
:100670000CC009F00EC00AF00FC013F016C00CF049
:100680000DC00DF019C00EF01AC00FF009C010F027
:100690000AC015F00DC0E9FF0EC0F3FF0F50B5EC16
:1006A00016F0166E1650D8B43ED00CC016F0176A6D
:1006B000161E171E1650171005E00CC016F00C067B
:1006C000165031E00DC0E9FF0EC0F3FF0F50B5EC3E
:1006D00016F0116E125010E01150E56EECEC15F0B2
:1006E000166EE652165004E01150166E169A02D09D
:1006F00011C016F016C011F01150E56E0250E56EF3
:100700000150E56E0050E56E49EC0EF0040EE12656
:100710000D2A02E30E4A0F2A104A152A1350D8B4A4
:10072000B9D71306B7D710C009F015C00AF0145096
:100730002BE010C00CF015C00DF013C00EF00E50E1
:100740001FE0200EE56E0250E56E0150E56E005090
:10075000E56E49EC0EF0040EE1260C4A0D2A0E0659
:10076000EED70B50E56E0250E56E0150E56E00507D
:10077000E56E49EC0EF0040EE126094A0A2A04D07F
:100780000CC009F00DC00AF0032A02E3044A052A4E
:100790007FEF00F00AC0F3FF0950E4CF1EF0E4CF72
:1007A0001DF0E4CF1CF0E4CF1BF0E4CF1AF0E4CF4F
:1007B00019F0E4CF18F0E4CF17F0E4CF16F0E4CF4F
:1007C00015F0E4CF14F0E4CF13F0E4CF12F0E4CF4F
:1007D00011F0E4CF10F0E4CF0FF0E4CF0EF0E4CF4F
:1007E0000DF0E4CF0CF0E4CF0BF0E4CF0AF0E4CF4F
:1007F00009F0E4CF08F0E4CF07F0E4CF06F0E4CF4F
:1008000005F0E4CF04F0E4CF03F0E4CF02F0E4CF4E
:1008100001F0E4CF00F0E4CFD9FF12003C4E4F20AE
:10082000464C4F41543E0000D350FC0BD36ED35086
:100830008F0B7009D36ED18004000F01676B0F011D
:10084000686B0F01696B0F016A6B0801036B08018C
:10085000046B0801056B0801066B08010F6B0F01A3
:10086000616B0F01626B0F01636B0F01646B0F0112
:10087000656B0F01666B0801106BD08E50EC15F0A4
:100880009F9A9F9819EC16F0000EE56E000EE56E2B
:10089000030EE56EE80EE56E49EC0BF0040EE12662
:1008A000000E026E140E016EFE0E006E0250E56E1A
:1008B0000150E56E0050E56E73EC12F0030EE12678
:1008C000B00EE56E030EE56E3C0EE56E000EE56EB5
:1008D00035EC12F0040EE1262EEC16F0BCEC15F00F
:1008E000006E005023E1010EE56EF9EC14F0E652C3
:1008F000000EE56E000EE56E030EE56EE80EE56E89
:1009000049EC0BF0040EE126000EE56EF9EC14F054
:10091000E652000EE56E000EE56E030EE56EE80E83
:10092000E56E49EC0BF0040EE126D8D7010EE56E1A
:10093000F9EC14F0E65291EC16F00801116F080E74
:10094000016E120E006E800E026E0250E56E0150B6
:10095000E56E0050E56E14EC10F0006E030EE1261B
:100960000050D8B43DD1080112510A0A05E008012F
:1009700012512E0A01E009D108010F6B000E016E21
:10098000E40E006E800E026E000E046EF90E036E11
:10099000800E056E0550E56E0450E56E0350E56E61
:1009A0000250E56E0150E56E0050E56EA0EC0AF0D5
:1009B000006E060EE1260050D8B4E3D004008B8A06
:1009C0000001F951006E0050610A01E196D000501B
:1009D000670A01E13CD00050730A05E000507A0A32
:1009E00001E169D0CAD0006A610E0024016E026A7A
:1009F0000F0E02220028036EF90E0324046E056A0E
:100A0000000E052204C0E9FF05C0EAFFEFCF04F0A5
:100A100001C0E9FF02C0EAFF04C0EFFF03C000F01D
:100A2000060E005CE1E3210E13EC17F0000E026EDF
:100A3000150E016E260E006E0250E56E0150E56E39
:100A40000050E56E73EC12F0030EE126C9D013C816
:100A500000F0016A000E046E150E036E2A0E026E7F
:100A60000F0E066E4E0E056E800E076E0150E56E7F
:100A70000050E56E0450E56E0350E56E0250E56EE1
:100A80000750E56E0650E56E0550E56EBFEC0DF0C3
:100A9000080EE1260F0E016E4E0E006E800E026EE5
:100AA0000250E56E0150E56E0050E56E73EC12F0F9
:100AB000030EE12695D07A0E13EC17F0000E026EAD
:100AC000150E016E260E006E0250E56E0150E56EA9
:100AD0000050E56E73EC12F0030EE126000EE56E99
:100AE000000EE56E000EE56E640EE56E49EC0BF04F
:100AF000040EE1260BEC17F073D0006A00C001F081
:100B0000026A000E056E150E046E320E036E0F0E95
:100B1000076E4E0E066E800E086E0F013251E56EA6
:100B20000F013151E56E0250E56E0150E56E055042
:100B3000E56E0450E56E0350E56E0850E56E075013
:100B4000E56E0650E56EBFEC0DF00A0EE1260F0EC5
:100B5000026E4E0E016E800E036E0350E56E025063
:100B6000E56E0150E56E73EC12F0030EE126002AEB
:100B7000080E005CD8A0C2D733D03F0E13EC17F09C
:100B80002FD03F0E13EC17F02BD0150E08010F5D80
:100B900010E2E40E08010F25006E016A000E01222A
:100BA00000C0E9FF01C0EAFF12C8EFFF08010F2BE8
:100BB00017D00001F86B08010F6B2B0E13EC17F028
:100BC000000E026E150E016E260E006E0250E56ECE
:100BD0000150E56E0050E56E73EC12F0030EE12655
:100BE000080113510801111904E013C811F807ECAA
:100BF00013F0006A016A026A0050E56E16EC15F007
:100C0000E6520AEC00F02EEC17F0036E0350FBE105
:100C1000310E0124036E0F0E0220046E22EC17F039
:100C2000056EF3CF06F003C0E9FF04C0EAFF05C07C
:100C3000EEFF06C0EFFF020E0126D8B0022A002AFE
:100C4000080E005CD9E37BD61200D9CFE5FFE1CFD7
:100C5000D9FF00C0E5FF01C0E5FF02C0E5FF03C00A
:100C6000E5FF04C0E5FF05C0E5FF06C0E5FF07C0DE
:100C7000E5FF020EDBCF00F0030EDBCF01F0040E28
:100C8000DBCF02F0050EDBCF03F0060EDBCF04F066
:100C9000070EDBCF05F0080EDBCF06F0090EDBCF29
:100CA00007F000500F016B6F01506C6F02506D6FB9
:100CB00003506E6F04500F016F6F0550706F065038
:100CC000716F0750726F0F016B510F017103F4CFF9
:100CD00001F0F3CF00F000500F01756F0150766FF7
:100CE0000F016B510F016F03F4CF01F0F3CF00F050
:100CF00000500F01736F0150746F0F016E510F019F
:100D00006F03F3CF00F00F01765100260050766F8D
:100D10000F016D510F017003F3CF00F00F017651F9
:100D200000260050766F0F016D510F016F03F4CF55
:100D300001F0F3CF00F00F0175510026765101222A
:100D40000050756F0150766F0F016C510F017003E9
:100D5000F4CF01F0F3CF00F00F017551002676516A
:100D600001220050756F0150766F0F016C510F0119
:100D70007103F3CF00F000500F017A6F0F016C5137
:100D80000F016F03F4CF01F0F3CF00F000500F011B
:100D9000786F0150796F0F016B510F017203F3CF20
:100DA00000F000500F017E6F0F016B510F017003B7
:100DB000F4CF01F0F3CF00F000500F017C6F015031
:100DC0007D6F0F01776B0F017B6B0F0177510F0167
:100DD0007325006E0F0178510F017421016E0F0110
:100DE00079510F017521026E0F017A510F017621A1
:100DF000036E0050736F0150746F0250756F035093
:100E0000766F0F017B510F017325006E0F017C512E
:100E10000F017421016E0F017D510F017521026ECA
:100E20000F017E510F017621036E03C0E9FF02C05E
:100E3000F4FF01C0F3FF0050E4CF07F0E4CF06F069
:100E4000E4CF05F0E4CF04F0E4CF03F0E4CF02F008
:100E5000E4CF01F0E4CF00F0E4CFD9FF12000000AE
:100E60002110422063308440A550C660E77008819D
:100E700029914AA16BB18CC1ADD1CEE1EFF1311214
:100E8000100273325222B5529442F772D6623993ED
:100E900018837BB35AA3BDD39CC3FFF3DEE3622464
:100EA000433420040114E664C774A44485546AA53D
:100EB0004BB528850995EEE5CFF5ACC58DD55336F4
:100EC000722611163006D776F6669556B4465BB78D
:100ED0007AA719973887DFF7FEE79DD7BCC7C448C4
:100EE000E5588668A7784008611802282338CCC9DD
:100EF000EDD98EE9AFF9488969990AA92BB9F55A54
:100F0000D44AB77A966A711A500A333A122AFDDB2C
:100F1000DCCBBFFB9EEB799B588B3BBB1AABA66C23
:100F2000877CE44CC55C222C033C600C411CAEED7C
:100F30008FFDECCDCDDD2AAD0BBD688D499D977E33
:100F4000B66ED55EF44E133E322E511E700E9FFFCC
:100F5000BEEFDDDFFCCF1BBF3AAF599F788F889182
:100F6000A981CAB1EBA10CD12DC14EF16FE1801066
:100F7000A100C230E3200450254046706760B98369
:100F80009893FBA3DAB33DC31CD37FE35EF3B102B6
:100F90009012F322D2323542145277625672EAB579
:100FA000CBA5A89589856EF54FE52CD50DC5E23406
:100FB000C324A01481046674476424540544DBA749
:100FC000FAB79987B8975FE77EF71DC73CD7D32656
:100FD000F2369106B01657667676154634564CD9D9
:100FE0006DC90EF92FE9C899E9898AB9ABA94458A6
:100FF000654806782768C018E1088238A3287DCBA9
:101000005CDB3FEB1EFBF98BD89BBBAB9ABB754AF5
:10101000545A376A167AF10AD01AB32A923A2EFD38
:101020000FED6CDD4DCDAABD8BADE89DC98D267C45
:10103000076C645C454CA23C832CE01CC10C1FEF88
:101040003EFF5DCF7CDF9BAFBABFD98FF89F176E95
:10105000367E554E745E932EB23ED10EF01ED9CF21
:10106000E5FFE1CFD9FF00C0E5FF01C0E5FF02C009
:10107000E5FF03C0E5FF04C0E5FF05C0E5FF06C0CE
:10108000E5FF07C0E5FF08C0E5FF09C0E5FF0AC0AE
:10109000E5FF0BC0E5FF0CC0E5FF020EDBCF00F063
:1010A000030EDBCF01F0040EDBCF02F0050EDBCF29
:1010B00003F0060EDBCF04F0070EDBCF05F0300E99
:1010C0000F01206F310E0F01216F320E0F01226FC1
:1010D000330E0F01236F340E0F01246F350E0F01F5
:1010E000256F360E0F01266F370E0F01276F380E52
:1010F0000F01286F390E0F01296F610E0F012A6F42
:10110000620E0F012B6F630E0F012C6F640E0F0127
:101110002D6F650E0F012E6F660E0F012F6F0F01E1
:10112000306B00C0E9FF01C0F3FF0250B5EC16F0D0
:10113000066E0650D8B460D00F0E086E200E076EF3
:10114000800E096E0650E56E0950E56E0850E56E9A
:101150000750E56EA9EC11F0066EF3CF07F0F4CF5F
:1011600008F0040EE126200E065E0F0E075A065008
:10117000100DF3CF06F00F0E086E200E076E800ED6
:10118000096E0050010F0A6E000E01200B6E000E5A
:1011900002200C6E0AC0E9FF0BC0F3FF0C50B5EC47
:1011A00016F00A6E0A50E56E0950E56E0850E56EBD
:1011B0000750E56EA9EC11F0076EF3CF08F0F4CFFD
:1011C00009F0040EE126200E075E0F0E085A0750A4
:1011D000062606C0E5FF03C0E9FF04C0F3FF055083
:1011E000E3EC16F0020E0026000E01220222032A72
:1011F00098E3044A052A95D7E4CF0CF0E4CF0BF02E
:10120000E4CF0AF0E4CF09F0E4CF08F0E4CF07F030
:10121000E4CF06F0E4CF05F0E4CF04F0E4CF03F030
:10122000E4CF02F0E4CF01F0E4CF00F0E4CFD9FF47
:101230001200D9CFE5FFE1CFD9FF00C0E5FF01C023
:10124000E5FF02C0E5FF03C0E5FF04C0E5FF05C000
:10125000E5FF06C0E5FF07C0E5FF08C0E5FF09C0E0
:10126000E5FF0AC0E5FF0BC0E5FF0CC0E5FF0DC0C0
:10127000E5FF0EC0E5FF0FC0E5FF020EDBCF00F07B
:10128000030EDBCF01F0040EDBCF02F0050EDBCF47
:1012900003F0060EDBCF04F0070EDBCF05F0080EDF
:1012A000DBCF06F0200E076E086A06C009F00A6A56
:1012B0000B6A0C6AE56AE56AE56A0950E56E035057
:1012C000E56E0250E56E0150E56E0050E56E96EC5D
:1012D0000CF00D6E080EE126300E0D263A0E0D5C58
:1012E00005E30D500E6E270E0E240D6EFF0E072621
:1012F0000822000E07240E6E0F0E08200F6E0EC07F
:10130000E9FF0FC0EAFF0DC0EFFF0C50E56E0B5078
:10131000E56E0A50E56E0950E56E0350E56E025029
:10132000E56E0150E56E0050E56E33EC0DF0006E99
:10133000F3CF01F0F4CF02F0E9CF03F0080EE1267D
:101340000050011002100310D8A4AFD707C000F05E
:1013500008C001F004C002F005C003F000C004F0B2
:1013600001C005F0004A012A000E04260F0E0522D6
:1013700004C0E9FF05C0EAFFEFCF04F002C0E9FFB7
:1013800003C0EAFF04C0EFFF024A032A000E015C1B
:1013900002E1200E005CE2E302C0E9FF03C0EAFFC5
:1013A000000EEF6AE4CF0FF0E4CF0EF0E4CF0DF0C3
:1013B000E4CF0CF0E4CF0BF0E4CF0AF0E4CF09F077
:1013C000E4CF08F0E4CF07F0E4CF06F0E4CF05F077
:1013D000E4CF04F0E4CF03F0E4CF02F0E4CF01F077
:1013E000E4CF00F0E4CFD9FF1200D8CFE5FFE0CF83
:1013F000E5FFE56EF3CFE5FFF4CFE5FFE9CFE5FFCD
:10140000EACFE5FFFACFE5FFFBCFE5FFD9CFE5FF58
:10141000E1CFD9FF00C0E5FF01C0E5FFF2A457D03E
:10142000FD0ED76ED66AF29491EC16F00801136F98
:101430000801076B0801086B610E08010725006EA3
:101440000F0E08010821016E00C0E9FF01C0EAFF8C
:10145000EFCF00F000500801105D15E2010E006EA4
:10146000016A0801075106E0E86CD89000360136A1
:10147000010FFCE3FF0EE56E0050E56EDCEC12F0B0
:10148000E652E65214D0010E006E016A08010751BF
:1014900006E0E86CD89000360136010FFCE3000E40
:1014A000E56E0050E56EDCEC12F0E652E652080103
:1014B000073F02D00801082B000E0801085D03E178
:1014C000060E0801075DD8A0B7D70801102BE4CF9E
:1014D00001F0E4CF00F0E4CFD9FFE4CFFBFFE4CF8D
:1014E000FAFFE4CFEAFFE4CFE9FFE4CFF4FFE4CF73
:1014F000F3FFE450E4CFE0FFE4CFD8FF10004F70DB
:10150000656E53746F6B6572207374617274696E6B
:10151000672E2E2E2073657269616C20776F726B57
:10152000696E670A0D000A0D000067253032780ADF
:101530000D00616425643A20253034780A0D0000DE
:10154000D9CFE5FFE1CFD9FF00C0E5FF01C0E5FF3E
:1015500002C0E5FF03C0E5FF04C0E5FF05C0E5FFED
:1015600006C0E5FF07C0E5FF08C0E5FF020EDBCFC0
:1015700000F0030EDBCF01F0040EDBCF02F0050E0E
:10158000DBCF03F0060EDBCF04F0070EDBCF05F058
:101590000F0E076E580E066E800E086E0850E56E30
:1015A0000750E56E0650E56E0250E56E0150E56E9F
:1015B0000050E56E2FEC08F0060EE1265FCF00F03C
:1015C000016A0050066E026A60CF00F0016A0050A6
:1015D0000226015006220F0E016E580E006E800E7C
:1015E000076E000EE56E000EE56E000EE56E000E55
:1015F000E56E000EE56E070EE56E0750E56E0150D4
:10160000E56E0050E56EF1EC0BF0006EF3CF01F0EB
:10161000090EE1260250001803E10650011801E00E
:1016200022D00550056E0450046E0350036E0F0E59
:10163000016E580E006E800E026E000EE56E070EF3
:10164000E56E0250E56E0150E56E0050E56E055006
:10165000E56E0450E56E0350E56ED2EC0EF0080E18
:10166000E126010E01D0E86AE4CF08F0E4CF07F0EC
:10167000E4CF06F0E4CF05F0E4CF04F0E4CF03F0CC
:10168000E4CF02F0E4CF01F0E4CF00F0E4CFD9FFE3
:101690001200D9CFE5FFE1CFD9FF00C0E5FF01C0BF
:1016A000E5FF02C0E5FF03C0E5FF04C0E5FF05C09C
:1016B000E5FF06C0E5FF07C0E5FF08C0E5FF09C07C
:1016C000E5FF0AC0E5FF0BC0E5FF0CC0E5FF0DC05C
:1016D000E5FF0EC0E5FF0FC0E5FF020EDBCF00F017
:1016E000030EDBCF01F0040EDBCF02F0050EDBCFE3
:1016F00003F067CF04F068CF05F069CF06F06ACF3A
:1017000007F004500F01675D086E05500F0168591E
:10171000096E06500F0169590A6E07500F016A5988
:101720000B6E08500C6E09500D6E0A500E6E0B5069
:101730000F6ED8800FAED8901CE30B50E56E0A50A8
:10174000E56E0950E56E0850E56EFF0EE56EFF0E82
:10175000E56EFF0EE56EFF0EE56E25EC06F00C6EF5
:10176000F3CF0DF0F4CF0EF0E9CF0FF0080EE12625
:1017700008D008C00CF009C00DF00AC00EF00BC074
:101780000FF003500F5C08E102500E5C05E10150C0
:101790000D5C02E100500C5CD8A0B3D7E4CF0FF091
:1017A000E4CF0EF0E4CF0DF0E4CF0CF0E4CF0BF07B
:1017B000E4CF0AF0E4CF09F0E4CF08F0E4CF07F07B
:1017C000E4CF06F0E4CF05F0E4CF04F0E4CF03F07B
:1017D000E4CF02F0E4CF01F0E4CF00F0E4CFD9FF92
:1017E0001200D9CFE5FFE1CFD9FF00C0E5FF01C06E
:1017F000E5FF02C0E5FF03C0E5FF04C0E5FF05C04B
:10180000E5FF06C0E5FF07C0E5FF08C0E5FF09C02A
:10181000E5FF0AC0E5FF0BC0E5FF0CC0E5FF020EC7
:10182000DBCF00F0030EDBCF01F0040EDBCF02F0C4
:10183000050EDBCF03F0060EDBCF04F0070EDBCF87
:1018400005F0080EDBCF06F0090EDBCF07F00A0E1D
:10185000DBCF08F003C009F004C00AF005C00BF0AC
:1018600006C00CF0FF0E03260422052206220950B2
:101870000A100B100C103AE00850096E00C0E9FF86
:1018800001C0F3FF0250B5EC16F00B6E002A02E324
:10189000014A022A0B50091AE56A0950E56EE56A09
:1018A000020EE56EBDEC10F0096EF3CF0AF0040EE7
:1018B000E1260B6A5E0E09260E0E0A22000E0B228E
:1018C00009C0F6FF0AC0F7FF0BC0F8FF0900F5CF0B
:1018D00009F00900F5CF0AF007500C6E0B6A0B50A7
:1018E0000918076E0C500A18086EB4D708C0F3FF29
:1018F0000750E4CF0CF0E4CF0BF0E4CF0AF0E4CFD4
:1019000009F0E4CF08F0E4CF07F0E4CF06F0E4CF2D
:1019100005F0E4CF04F0E4CF03F0E4CF02F0E4CF2D
:1019200001F0E4CF00F0E4CFD9FF1200D9CFE5FFFA
:10193000E1CFD9FF00C0E5FF01C0E5FF02C0E5FF30
:1019400003C0E5FF04C0E5FF05C0E5FF06C0E5FFF5
:1019500007C0E5FF08C0E5FF09C0E5FF0AC0E5FFD5
:10196000020EDBCF00F0030EDBCF01F0040EDBCF65
:1019700002F0050EDBCF03F0060EDBCF04F0070EFE
:10198000DBCF05F0080EDBCF06F0090EDBCF07F04A
:10199000086A045005100610071005E1E968F468AC
:1019A000F368E86847D0096A0750800BE8440A6E7C
:1019B0000A501BE104500426053606360736075048
:1019C000035C08E10650025C05E10550015C02E1A0
:1019D0000450005C06E2D890073206320532043229
:1019E00004D0092A09C008F0DFD70750035C08E1DA
:1019F0000650025C05E10550015C02E10450005C08
:101A000008E30450005E0550015A0650025A075080
:101A1000035AD890073206320532043208C009F062
:101A200008060950E2E103C0E9FF02C0F4FF01C06B
:101A3000F3FF0050E4CF0AF0E4CF09F0E4CF08F060
:101A4000E4CF07F0E4CF06F0E4CF05F0E4CF04F0F4
:101A5000E4CF03F0E4CF02F0E4CF01F0E4CF00F0F4
:101A6000E4CFD9FF1200D9CFE5FFE1CFD9FF00C005
:101A7000E5FF01C0E5FF02C0E5FF03C0E5FF04C0CC
:101A8000E5FF05C0E5FF06C0E5FF07C0E5FF08C0AC
:101A9000E5FF09C0E5FF0AC0E5FF0BC0E5FF0CC08C
:101AA000E5FF0DC0E5FF020EDBCF00F0030EDBCF3C
:101AB00001F0040EDBCF02F0050EDBCF03F0060EC3
:101AC000DBCF04F0070EDBCF05F0080EDBCF06F00E
:101AD000090EDBCF07F0086A096A0A6A0B6A200E52
:101AE0000C6E0350800BE8440D6E0050002601364A
:101AF000023603360850082609360A360B360D50D2
:101B0000D8A4088007500B5C08E106500A5C05E188
:101B10000550095C02E10450085C09E30450085ECA
:101B20000550095A06500A5A07500B5A00800C2ECD
:101B3000D8D703C0E9FF02C0F4FF01C0F3FF005093
:101B4000E4CF0DF0E4CF0CF0E4CF0BF0E4CF0AF0DB
:101B5000E4CF09F0E4CF08F0E4CF07F0E4CF06F0DB
:101B6000E4CF05F0E4CF04F0E4CF03F0E4CF02F0DB
:101B7000E4CF01F0E4CF00F0E4CFD9FF1200D9CFD9
:101B8000E5FFE1CFD9FF00C0E5FF01C0E5FF02C0DE
:101B9000E5FF03C0E5FF04C0E5FF05C0E5FF050E56
:101BA000D924006E000EDA20016E800E026E030E44
:101BB0000026000E0122022206C0E5FF07C0E5FF55
:101BC00008C0E5FF020EDBCF06F0030EDBCF07F007
:101BD000040EDBCF08F00850056E0750046E065067
:101BE000036EE4CF08F0E4CF07F0E4CF06F0025034
:101BF000E56E0150E56E0050E56E070EDBCFE5FFA8
:101C0000060EDBCFE5FF050EDBCFE5FF0550E56EE9
:101C10000450E56E0350E56E0EEC00F0006EF3CF5D
:101C200001F0090EE12606C0E5FF07C0E5FF08C088
:101C3000E5FF020EDBCF06F0030EDBCF07F0040E4C
:101C4000DBCF08F000500624026E01500720036E1F
:101C5000E86A0820E4CF08F0E4CF07F0E4CF06F00C
:101C6000E56A02C0E9FF03C0F3FFE3EC16F001C030
:101C7000F3FF0050E4CF05F0E4CF04F0E4CF03F02D
:101C8000E4CF02F0E4CF01F0E4CF00F0E4CFD9FFDD
:101C90001200D9CFE5FFE1CFD9FF00C0E5FF01C0B9
:101CA000E5FF02C0E5FF03C0E5FF04C0E5FF05C096
:101CB000E5FF06C0E5FF07C0E5FF020EDBCF00F041
:101CC000030EDBCF01F0040EDBCF02F0050EDBCFFD
:101CD00003F002C006F00650046E800A33E100C033
:101CE000E9FF01C0F3FF025087EC15F0056EF3CF5A
:101CF00006F0F4CF07F003C0E5FF05C0E9FF06C01A
:101D0000F3FF0750E3EC16F000C0E9FF01C0F3FF5A
:101D1000025087EC15F0056EF3CF06F0F4CF07F014
:101D2000052A02E3064A072A05C0E5FF06C0F4FFBC
:101D300007C0F6FF00C0E9FF01C0F3FF0250C6EC88
:101D400016F01DD004AA1BD0047A045004E10350FD
:101D500006EC00F014D00450010A04E1035002EC38
:101D600000F00DD004500F0A04E1035041EC17F0CD
:101D700006D004500E0A03E1035032EC17F0E4CF12
:101D800007F0E4CF06F0E4CF05F0E4CF04F0E4CFB1
:101D900003F0E4CF02F0E4CF01F0E4CF00F0E4CFB1
:101DA000D9FF1200D9CFE5FFE1CFD9FF00C0E5FF91
:101DB00001C0E5FF02C0E5FF03C0E5FF04C0E5FF89
:101DC00005C0E5FF06C0E5FF07C0E5FF08C0E5FF69
:101DD00009C0E5FF0AC0E5FF0BC0E5FF0CC0E5FF49
:101DE000020EDBCF00F0030EDBCF01F0040EDBCFE1
:101DF00002F0050EDBCF03F0060EDBCF04F0070E7A
:101E0000DBCF05F0080EDBCF06F0090EDBCF07F0C5
:101E100002500A6E0150096E0050086E06C00BF0A9
:101E200007C00CF0FF0E062607220B500C101AE01C
:101E300003C0E9FF04C0F3FF0550B5EC16F00B6ECC
:101E4000032A02E3044A052A0BC0E5FF08C0E9FFA4
:101E500009C0F3FF0A50E3EC16F0082ADFE3094A51
:101E60000A2ADCD702C0F4FF01C0F3FF0050E4CF20
:101E70000CF0E4CF0BF0E4CF0AF0E4CF09F0E4CFAC
:101E800008F0E4CF07F0E4CF06F0E4CF05F0E4CFAC
:101E900004F0E4CF03F0E4CF02F0E4CF01F0E4CFAC
:101EA00000F0E4CFD9FF1200D9CFE5FFE1CFD9FF91
:101EB00000C0E5FF01C0E5FF02C0E5FF03C0E5FF8C
:101EC00004C0E5FF05C0E5FF06C0E5FF020EDBCF5D
:101ED00000F0030EDBCF01F0040EDBCF02F0050EA5
:101EE000DBCF03F0060EDBCF04F0070EDBCF05F0EF
:101EF000080EDBCF06F0D88003AED89015E306506D
:101F00000A0A12E104C0E9FF05C0EAFF2D0EEF6ED8
:101F1000044A052A031E021E011E006C05E1012A67
:101F200003E1022AD8B4032A0650E56E0550E56E97
:101F30000450E56E0350E56E0250E56E0150E56E0B
:101F40000050E56E19EC09F0070EE126E4CF06F02B
:101F5000E4CF05F0E4CF04F0E4CF03F0E4CF02F0E7
:101F6000E4CF01F0E4CF00F0E4CFD9FF1200D9CFE5
:101F7000E5FFE1CFD9FF00C0E5FF01C0E5FF02C0EA
:101F8000E5FF03C0E5FF04C0E5FF05C0E5FF06C0AF
:101F9000E5FF020EDBCF00F0030EDBCF01F0040EF5
:101FA000DBCF02F0050EDBCF03F0046A056A0350B5
:101FB000800BE844066E065011E1025002260336FB
:101FC0000350015C02E10250005C04E2D89003324D
:101FD000023204D0052A05C004F0E9D70350015CA1
:101FE00002E10250005C04E30250005E0350015A1B
:101FF000D8900332023204C005F004060550EEE129
:1020000001C0F3FF0050E4CF06F0E4CF05F0E4CFC9
:1020100004F0E4CF03F0E4CF02F0E4CF01F0E4CF2A
:1020200000F0E4CFD9FF1200D9CFE5FFE1CFD9FF0F
:1020300000C0E5FF01C0E5FF02C0E5FF03C0E5FF0A
:1020400004C0E5FF020EDBCF00F0030EDBCF01F092
:10205000040EDBCF02F0BCEC15F0036E03502DE054
:1020600005C803F006C804F00801053F02D00801C6
:10207000062B000EE56E640EE56E0450E56E03500F
:10208000E56EB7EC0FF0036EF3CF04F0040EE1261B
:10209000800E0326000E042203C0E9FF04C0EAFFFD
:1020A000EFCF03F003C0E5FF00C0E9FF01C0F3FF7D
:1020B0000250E3EC16F0010E01D0E86AE4CF04F020
:1020C000E4CF03F0E4CF02F0E4CF01F0E4CF00F07E
:1020D000E4CFD9FF1200D9CFE5FFE1CFD9FF00C08F
:1020E000E5FF01C0E5FF02C0E5FF020EDBCF00F017
:1020F000030EDBCF01F000AC06D0020EE56E59EC0A
:1021000013F0E65205D0010EE56E59EC13F0E652DD
:102110000138E8441F0B026E0250E56EA5EC13F087
:10212000E6523F0E00160050E56E81EC13F0E652C9
:10213000EEEC16F0EEEC16F0026E0050E56E81EC5F
:1021400013F0E652070E0116010E006E015005E075
:10215000E86CD8900036010FFDE3005002120250E7
:10216000E56EC8EC13F0E652E4CF02F0E4CF01F0E4
:10217000E4CF00F0E4CFD9FF1200D9CFE5FFE1CFE3
:10218000D9FF00C0E5FF01C0E5FF02C0E5FF03C0C5
:10219000E5FF020EDBCF00F0030EDBCF01F0040EF3
:1021A000DBCF02F0050EDBCF03F000500801096F12
:1021B00001500A6F025008010B6F03500C6F0801A9
:1021C000095108010B03F4CF01F0F3CF00F00050E8
:1021D00008010D6F01500E6F0801095108010C0331
:1021E000F3CF00F008010A5108010B03F3CF01F00F
:1021F0000150002608010E51002600500E6F0EC837
:10220000F3FF0D51E4CF03F0E4CF02F0E4CF01F08F
:10221000E4CF00F0E4CFD9FF1200D8CFE5FFE0CF44
:10222000E5FFE56EF3CFE5FFF4CFE5FFE9CFE5FF8E
:10223000EACFE5FFFACFE5FFFBCFE5FFD9CFE5FF1A
:10224000E1CFD9FF00C0E5FF9EA010D0FE0ECF6EFB
:10225000C80ECE6E9E900F01672B08E30F01682B0E
:1022600005E30F01693F02D00F016A2B2AEC17F03A
:10227000006E00500BE06AEC16F0006E0050E56E48
:10228000F4EC11F0E652005013EC17F0E4CF00F03C
:10229000E4CFD9FFE4CFFBFFE4CFFAFFE4CFEAFFBE
:1022A000E4CFE9FFE4CFF4FFE4CFF3FFE450E4CF61
:1022B000E0FFE4CFD8FF1000D9CFE5FFE1CFD9FF91
:1022C00000C0E5FF01C0E5FF02C0E5FF030EE56EBB
:1022D00059EC13F0E652006A0050E56EA5EC13F0DD
:1022E000E652000EE56E81EC13F0E652000EE56E4C
:1022F00042EC16F0E652000EE56EA2EC14F0E65247
:10230000010EE56EBFEC14F0E652400E016EE9ECF2
:1023100013F00000000000000000000000000000BA
:1023200000000150026E0204016E0150F0E1002A2B
:10233000080E005CD1E3010EE56E59EC13F0E65295
:10234000E4CF02F0E4CF01F0E4CF00F0E4CFD9FF16
:102350001200D9CFE5FFE1CFD9FF00C0E5FF01C0F2
:10236000E5FF02C0E5FF03C0E5FF04C0E5FF020E84
:10237000DBCF00F0030EDBCF01F0040EDBCF02F069
:10238000050EDBCF03F000C0E9FF01C0F3FF0250F0
:10239000B5EC16F0046E045008E00450031805E094
:1023A000002A02E3014A022AEED700C0E9FF01C079
:1023B000F3FF0250B5EC16F0031806E102C0F4FF7B
:1023C00001C0F3FF005003D0F46AF36AE86AE4CF77
:1023D00004F0E4CF03F0E4CF02F0E4CF01F0E4CF67
:1023E00000F0E4CFD9FF1200D9CFE5FFE1CFD9FF4C
:1023F00000C0E5FF01C0E5FF02C0E5FF020EDBCF34
:1024000000F0BCEC15F0016E0150640A24E003C832
:1024100001F004C802F00801033F02D00801042BB8
:10242000000EE56E640EE56E0250E56E0150E56E3D
:10243000B7EC0FF0016EF3CF02F0040EE126800E30
:102440000126000E022201C0E9FF02C0EAFF00C01F
:10245000EFFF010E01D0E86AE4CF02F0E4CF01F013
:10246000E4CF00F0E4CFD9FF1200D9CFE5FFE1CFF0
:10247000D9FF00C0E5FF01C0E5FF02C0E5FF03C0D2
:10248000E5FF020EDBCF00F0030EDBCF01F0040E00
:10249000DBCF02F0050EDBCF03F0C26A0F0E001691
:1024A0000044E844FC0BC26E3F0E0216300E0314CB
:1024B0000210C16E800E0314006E3F0E0116015013
:1024C0000010C06E03AC03D09E9C9D8CF28CC28029
:1024D000E4CF03F0E4CF02F0E4CF01F0E4CF00F06A
:1024E000E4CFD9FF1200D9CFE5FFE1CFD9FF00C07B
:1024F000E5FF01C0E5FF02C0E5FF03C0E5FF020EF6
:10250000DBCF00F0030EDBCF01F0040EDBCF02F0D7
:1025100026EC17F0036E0350FBE100C0E9FF01C099
:10252000F3FF0250B5EC16F013EC17F000C0E9FF12
:1025300001C0F3FF0250B5EC16F0036E002A02E36F
:10254000014A022A0350E4E1E4CF03F0E4CF02F0B1
:10255000E4CF01F0E4CF00F0E4CFD9FF1200D9CFEF
:10256000E5FFE1CFD9FF00C0E5FF020EDBCF00F0B1
:10257000010EE56E4BEC14F0E652010EE56E68ECD0
:1025800014F0E652000EE56EA2EC14F0E652000ED6
:10259000E56EBFEC14F0E652010E00163E0E00127E
:1025A0000050E56E42EC16F0E652E9EC13F0E4CF91
:1025B00000F0E4CFD9FF1200D9CFE5FFE1CFD9FF7A
:1025C00000C0E5FF01C0E5FF020EDBCF00F0030E07
:1025D000DBCF01F03F0E001600500116956A015046
:1025E00006E000500801141314C88CFF06D0001E2A
:1025F00000500801141714C88CFF898E899E8C6ABC
:10260000E4CF01F0E4CF00F0E4CFD9FF1200D9CF3E
:10261000E5FFE1CFD9FF000EE56EF9EC14F0E652CC
:10262000000EE56E000EE56E000EE56EC80EE56E5E
:1026300049EC0BF0040EE126010EE56EF9EC14F006
:10264000E652000EE56E000EE56E000EE56EC80E59
:10265000E56E49EC0BF0040EE126E4CFD9FF120041
:10266000D9CFE5FFE1CFD9FF000EE56E000EE56E94
:10267000000EE56E010EE56E49EC0BF0040EE1264E
:10268000000EE56E85EC14F0E652000EE56E000ECD
:10269000E56E000EE56E010EE56E49EC0BF0040EE2
:1026A000E126010EE56E85EC14F0E652E4CFD9FF89
:1026B0001200D9CFE5FFE1CFD9FF00C0E5FF020E40
:1026C000DBCF00F000A006D0010EE56E4BEC14F05D
:1026D000E65205D0000EE56E4BEC14F0E65200A277
:1026E00006D0010EE56E68EC14F0E65205D0000E3F
:1026F000E56E68EC14F0E652E4CF00F0E4CFD9FFC9
:102700001200D9CFE5FFE1CFD9FF00C0E5FF020EEF
:10271000DBCF00F06CEC15F0000EE56EBFEC14F0B2
:10272000E652000EE56EA2EC14F0E6523F0E0016E3
:10273000008C0050E56E42EC16F0E652E9EC13F026
:10274000E4CF00F0E4CFD9FF1200D9CFE5FFE1CF0D
:10275000D9FF00C0E5FF020EDBCF00F06CEC15F0F6
:10276000000EE56EBFEC14F0E652000EE56EA2EC32
:1027700014F0E652B80E00120050E56E42EC16F06E
:10278000E652E9EC13F0E4CF00F0E4CFD9FF1200F9
:10279000D9CFE5FFE1CFD9FF00C0E5FF020EDBCFC7
:1027A00000F06CEC15F0010EE56EBFEC14F0E65293
:1027B000000EE56EA2EC14F0E6520050E56E42EC1D
:1027C00016F0E652E9EC13F0E4CF00F0E4CFD9FFC5
:1027D0001200D9CFE5FFE1CFD9FF010EE56EDCECA9
:1027E00014F0E652000000000000000000000000AD
:1027F00000000000000EE56EDCEC14F0E652000074
:102800000000000000000000000000000000E4CF15
:10281000D9FF1200D9CFE5FFE1CFD9FF010EE56E58
:10282000F9EC14F0E6520801166B000EE56E4BEC65
:1028300014F0E652000EE56E68EC14F0E65230EC4F
:1028400013F0010EE56EAFEC12F0E6525CEC11F005
:10285000E4CFD9FF1200E8AE0AD0F3CFEAFFEE5082
:10286000EECFF3FFEECFF4FFEECFE9FF1200E8BCAE
:102870003DEF17F0E9CFF6FFF3CFF7FFF86E090051
:10288000F5500900F5CFF3FF0900F5CFF4FF09007B
:10289000F5CFE9FF1200D9CFE5FFE1CFD9FF00C0A6
:1028A000E5FF020EDBCF00F0956A005005E008015D
:1028B000168B16C88CFF04D00801169B16C88CFF17
:1028C000898C899C8C6AE4CF00F0E4CFD9FF120098
:1028D000D9CFE5FFE1CFD9FF00C0E5FF020EDBCF86
:1028E00000F0956A005005E00801168916C88CFFB3
:1028F00004D00801169916C88CFF898C899C8C6AB3
:10290000E4CF00F0E4CFD9FF1200D9CFE5FFE1CF4B
:10291000D9FF00C0E5FF020EDBCF00F0956A005042
:1029200005E00801168716C88CFF04D00801169729
:1029300016C88CFF898C899C8C6AE4CF00F0E4CFA8
:10294000D9FF1200D9CFE5FFE1CFD9FF00C0E5FFE5
:10295000020EDBCF00F0956A005005E008011685F5
:1029600016C88CFF04D00801169516C88CFF898CF8
:10297000899C8C6AE4CF00F0E4CFD9FF1200D9CF54
:10298000E5FFE1CFD9FF00C0E5FF020EDBCF00F08D
:10299000956A005005E00801168316C88CFF04D024
:1029A0000801169316C88CFF898C899C8C6AE4CF29
:1029B00000F0E4CFD9FF1200D9CFE5FFE1CFD9FF76
:1029C00000C0E5FF020EDBCF00F0956A005005E085
:1029D0000801168116C88CFF04D00801169116C88C
:1029E0008CFF898C899C8C6AE4CF00F0E4CFD9FFFE
:1029F0001200D9CFE5FFE1CFD9FF00C0E5FF020EFD
:102A0000DBCF00F0956A005005E00801168F16C86C
:102A10008CFF04D00801169F16C88CFF898C899CF6
:102A20008C6AE4CF00F0E4CFD9FF1200D9CFE5FFE4
:102A3000E1CFD9FF00C0E5FF01C0E5FF020EDBCF0B
:102A400000F0C250016EC30E01160F0E00160044B6
:102A5000E844FC0B0110C26EE4CF01F0E4CF00F0BB
:102A6000E4CFD9FF1200F2CFF6FFF29EA69EA69CFD
:102A7000E9CFA9FFF3CFAAFFA680A850A94AAA2AA6
:102A8000A680A8CFF3FFA94AAA2AA680A8CFF4FF60
:102A9000A94AAA2AA680A8CFEAFFF6BEF28E1200A3
:102AA000D9CFE5FFE1CFD9FFD58ED590D592D5947A
:102AB000D59CD59AD596F184F28AF284CD80CD8EBC
:102AC000CD92CD96CD88CD8A9F909D809E80F28CB0
:102AD000F28EE4CFD9FF1200D9CFE5FFE1CFD9FFC5
:102AE00000000000000000000000000000000000E6
:102AF000000EE56E000EE56E000EE56E0A0EE56E48
:102B000049EC0BF0040EE126E4CFD9FF1200E8AE49
:102B100008D0F3CFEAFFEE50EECFF3FFEECFF4FF95
:102B20001200E8BC3BEF17F0E9CFF6FFF3CFF7FF59
:102B3000F86E0900F5500900F5CFF3FF0900F5CF55
:102B4000F4FF1200F2CFEAFFF29EA69EA69CA68496
:102B5000E9CFA9FFF3CFAAFFE4CFA8FF02EC17F05B
:102B6000F4CFA8FF02EC17F0F6CFA8FF02EC17F0A5
:102B7000A694EABEF28E1200D9CFE5FFE1CFD9FFCD
:102B800000C0E5FF01C0E5FF08010351006E080128
:102B90000551016E0150005E0050E4CF01F0E4CF1A
:102BA00000F0E4CFD9FF1200F2CFF6FFF29EA69E0E
:102BB000A69CE9CFA9FFF3CFAAFFA680A850A94AF7
:102BC000AA2AA680A8CFF3FFA94AAA2AA680A8CF3E
:102BD000F4FFF6BEF28E1200D9CFE5FFE1CFD9FFA8
:102BE00000C0E5FF020EDBCF00F0610E005C05E3E4
:102BF0007B0E005C02E2010E01D0E86AE4CF00F037
:102C0000E4CFD9FF1200E8AE06D0F3CFEAFFEE50D2
:102C1000EECFF3FF1200E8BC39EF17F0E9CFF6FF73
:102C2000F3CFF7FFF86E0900F5500900F5CFF3FF79
:102C30001200D9CFE5FFE1CFD9FF670EAF6EAC84AC
:102C4000AC98B886AB8E9D989F989D8A9F9AAC9CB5
:102C5000AB9CAB88AC8AE4CFD9FF1200D9CFE5FF9B
:102C6000E1CFD9FF956A92988988929E899E080142
:102C7000146B929C899C94948B94949A8B9AE4CF35
:102C8000D9FF1200D9CFE5FFE1CFD9FF00C0E5FFA2
:102C9000020EDBCF00F0956A00C08CFF8B848B9412
:102CA0008C6AE4CF00F0E4CFD9FF1200D9CFE5FF62
:102CB000E1CFD9FF000EE56E000EE56E000EE56E69
:102CC0000A0EE56E49EC0BF0040EE126010EE4CF8E
:102CD000D9FF1200F00E08011715176FABAC04D026
:102CE0001791ABA001D01781ABA402D008011785C2
:102CF000ABA202D008011787AE501200F2CFF6FF48
:102D0000F29EA69EA69CE9CFA9FFF3CFAAFFA680BC
:102D1000A850A94AAA2AA680A8CFF3FFF6BEF28E31
:102D20001200D9CFE5FFE1CFD9FF00C0E5FFFF0ECC
:102D3000956E899883CF00F089880050E4CF00F029
:102D4000E4CFD9FF1200F2CFEAFFF29EA69EA69C26
:102D5000A684E9CFA9FFF3CFAAFFE4CFA8FF02EC36
:102D600017F0A694EABEF28E1200E8AE04D0F3CFBC
:102D7000EAFFEE501200E8BC37EF17F0E9CFF6FF9C
:102D8000F3CFF7FFF86E0900F5501200E8AE09D056
:102D9000F3CFEAFFE4CFEEFFF4CFEEFFF6CFEEFF86
:102DA0001200E8BC3FEF17F01200F2CFF6FFF29EE0
:102DB000A69EA69CE9CFA9FFF3CFAAFFA680A850A4
:102DC000F6BEF28E1200E8AE05D0F3CFEAFFE4CFF4
:102DD000EEFF1200E8BC35EF17F01200D9CFE5FF87
:102DE000E1CFD9FFE9EC13F0E86AE4CFD9FF120094
:102DF00017EEFFF027EEFFF0F86AA68EA69C14EC03
:102E000004F0FFD7550EA76EAA0EA76EA682A6B233
:102E1000FED7A94AAA2AD9CFE5FFE1CFD9FFFF0003
:102E2000E4CFD9FF1200ACAC04D0AC90080117B3CA
:102E3000AC80AD6E1200D9CFE5FFE1CFD9FFE4CF72
:102E4000D9FF1200C4CFF3FFC3501200000EACA292
:102E5000010F1200000E9EBA010F1200000EC2B246
:102E6000010F1200E8CF7FFF1200A3EF16F0D5EF9D
:102E700016F07EEF16F0D4EF15F033EF15F0A2EF59
:042E800015F0120037
:020000040030CA
:0300010008191AC1
:020005008180F8
:00000001FF
